:1000000004298030A100FE30A4200130A4207530E6
:10001000A7003030CF28A101A117AF00FE30A420E7
:100020002F08A428A401AA00AB01A01124080319D9
:10003000A0151030A3000301AA0DAB0D0318013069
:1000400045202308031D1B280800A401AA00AB01BA
:10005000A01124080319A0150530A3002730A9001A
:1000600010303E200330A900E8303E20A901643062
:100070003E20A9010A303E202A084528A8002B0866
:10008000A7002A08A600E3202608A600A303031958
:10009000A011240803194F28230203185628260804
:1000A000031DA011A0195628303EA4280800AD0059
:1000B000051085108316051085100F3086058312F4
:1000C0002D08A01881283E30A7008030CF20333083
:1000D000AC0095201330A7008830CF2095206430E5
:1000E000CE2095206430CE202230AC0095202830E0
:1000F00080200C30802006308020A0142D0881281C
:100100002014AC00201C8F288510033C031C94286D
:1001100094200530A700DC30CF2003140800201401
:10012000FE3C0319A2288514201C201005140F3052
:1001300086052C08F03986040510AC0E2018952889
:100140003230CE202D08FF28A11B572883169B0094
:1001500083161C141A089B0AFF2883169A001C1584
:1001600055309D00AA309D009C149C18B5281C1188
:100170009B0AFF2883178001840AFF3E031DBB28CA
:10018000FF28A901A800FF30A807031CA907031C2A
:10019000FF280330A700E530CF20C328A701F63E93
:1001A000A600A709031CDA28FE300000A6070318E2
:1001B000D528A6070000A70FD42800002618E0289D
:1001C0002618E2280800AB01AA011030AC00270D68
:1001D000AA0DAB0D2808AA022908031C290FAB029F
:1001E0000318F9282808AA0729080318290FAB07BC
:1001F0000310A60DA70DAC0BE7282608FF288313D4
:100200008312031300000800A00107309F00F130A3
:1002100083168500FF3086008113831285018601D5
:10022000203084006030BB20A03084005030BB20E0
:10023000203084003030BA200130A900F430C220D0
:1002400001204930572052305720203057205A3053
:100250005720653057206E30572064305720653066
:10026000572072305720203057204E3057204C30C6
:10027000572020305720563057202D30572031300E
:1002800057208030A100C0300B20773057205720F6
:1002900057202E3057207030572069305720633058
:1002A0005720623057206130572073305720693013
:1002B0005720633057202E3057206E3057206C3037
:1002C00057200730A900D030C2208618A829012065
:1002D000503057204F30572052305720543057203D
:1002E000423057202E3057203130572020305720B1
:1002F0006D3057206130572067305720203057200D
:100300006E305720753057208030A100C0300B2050
:100310006E30572069305720653057207430572091
:10032000203057206C3057206130572057206730DD
:100330005720203057207A305720693057206A30B4
:1003400057206E3057208618A629A3293230C120A5
:100350000120493057204E30572053305720543019
:100360005720453057204C3057203D3057204B30D8
:10037000572065305720753057207A305720653028
:1003800057208030A100C0300B205A305720453014
:1003900057204E305720443057203D30572056309C
:1003A0005720653057207230572064305720653011
:1003B0005720723057202030572067305720613047
:1003C000572057206E3057200301A620A50025088E
:1003D000013A013903193211031D3215061D352A60
:1003E0000530C120030132190130013A03193211DD
:1003F000031D32158D300B20A101321D062A52300B
:10040000572043305720353057200C2A5230572080
:10041000433057203630572006180F2A0C2A030184
:1004200006180130B1000301061901303105031926
:100430001A2A0F2A8030A100C5300B2042305720E5
:10044000653057207630572065305720733057205D
:100450007430572069305720673057206530572057
:100460006E30572020305720EE290619382A352AB9
:100470000301A620A50025083219013C0319472ACB
:1004800083169B010301831232190130AD20321D06
:10049000512A7F30B6001F30B7000130A620B900C6
:1004A000582AFF30B600FF30B7000230A620B9004E
:1004B0000130B30032145D22B22A8030A1008030B6
:1004C0000B205330572079305720733057203A3063
:1004D00057203908252020305720572057208030BA
:1004E000A10088300B2039081220203057205720D7
:1004F000572057205720572057208030A100C03068
:100500000B20433057206F3057206D3057203A3042
:10051000572033082520203057205720572080307F
:10052000A100C8300B20330812202030572057205C
:100530005720572057205720572008000130061811
:100540000301B10001303A02030103180130310503
:100550000319B12ABA030230C1200619B02AB12A00
:100560009E2A0800030106190130B1000301061894
:10057000013031050319C02AFA30B800B211B22A8D
:100580000530C120030106190130B100030106182E
:10059000013031050319CD2AB22A0618302B06196D
:1005A000D22A5A2BFA303802031DF52AC830BB0074
:1005B000013006180301B10001303B0203010318AA
:1005C000013031050319E82A0530C120BB03D82AC0
:1005D00001303B020318F52A030132180130013AB9
:1005E00003193210031D3214B215321C0A2B86185F
:1005F000022BB214370839020318002BB90A012B59
:10060000B901092B360833020318082BB30A092B4A
:10061000B3011C2B8618152BB214B9080319122B21
:10062000B903142B3708B9001C2BB30803191A2B74
:10063000B3031C2B3608B3005D22B21D2F2B3808E4
:10064000BA009E22FA303802031D292BFA30BA0074
:100650009E220B303802031C2F2B0A30B802592B74
:100660000619592BB21C442BB210321D3E2B0130FF
:1006700083169B0083123908AD20442B0230831669
:100680009B0083123908AD200301321A0130013A70
:1006900003193212031D32160619592B321D522B23
:1006A0007723532BCE230618562B5A2B5230C120BA
:1006B0004C2BB22A01204830572065305720723029
:1006C00057207330572074305720613057207230D4
:1006D000572074305720013006180301B100013053
:1006E0000619030131040319762B6B2B0D29B02356
:1006F000331FB023331BAD23321AB023321EAD2378
:10070000391AB023391EAD23B919B023B91DAD2351
:100710003919B023391DAD23B918B023B91CAD2345
:100720003918B023391CAD23B31AB023B31EAD233F
:10073000331AB023331EAD23B319B023B31DAD2339
:100740003319B023331DAD23B318B023B31CAD232D
:100750003318B023331CAD230800BE23B323080095
:10076000B323BE230800FF30B500000000000000E6
:10077000000000000000B50BB52B08002030B400CD
:1007800000000F30B500B50BC32B05150530B500C3
:10079000B50BC82B0511B40BC02B08003224322432
:1007A00032243224322432242B242B2428242524BE
:1007B00025242524321E3224321E32242B242B24BD
:1007C000321A3224321A3224B91B2824B91F2524A4
:1007D000391B2824391F2524B91A2824B91E252499
:1007E000391A2824391E2524B9192824B91D25248D
:1007F00039192824391D2524B9182824B91C252481
:1008000039182824391C2524B31B2824B31F252478
:10081000331B2824331F2524B31A2824B31E252470
:10082000331A2824331E2524B3192824B31D252464
:1008300033192824331D2524B3182824B31C252458
:1008400033182824331C252408002B2432240800C4
:1008500032242B240800E130B50000000000B50B65
:100860002D2C08001030B40000000F30B500B50B7F
:10087000372C05150530B500B50B3C2C0511B40B14
:04088000342C08000C
:02400E00223F4F
:06420000000000000000B8
:00000001FF
